:1000000012C039C385C31895189518951895189579
:10001000F0C2189518951895189518951895189573
:100020001895189518958FE58DBFC0EEE8E64E2E11
:1000300084E08EBFD3E0F3E05F2EA89584B7082E4E
:10004000877F84BF88E1992781BD91BDEEEFF3E002
:10005000A0E6B0E088278D933197E9F789E189B967
:1000600080E080BD88E18AB90E942C09662480E086
:100070008FBD84E08EBD8EEE95E89DBD8CBD79B7B9
:10008000746079BFBB9A85E685BD79B7706479BF26
:1000900062D984E690E0DFD98CE0B1D9E4EBF0E0FE
:1000A00080E4ADD958E0C895802DA3D931965A95F2
:1000B000D1F704C01010101010101E1EE4EDF0E077
:1000C00088E49DD958E0C895802D93D931965A95EA
:1000D000D1F704C00F090A0C08080808E4EFF0E0A3
:1000E00080E58DD958E0C895802D83D931965A95F1
:1000F000D1F704C01C04202020202020E4E1F1E0FE
:1001000088E57DD958E0C895802D73D931965A95E8
:10011000D1F704C01C04040E11110E04E4E3F1E055
:1001200080E66DD958E0C895802D63D931965A95EF
:10013000D1F704C00404040420202020E4E5F1E009
:1001400088E65DD958E0C895802D53D931965A95E7
:10015000D1F704C00404040408101020E4E7F1E01F
:1001600080E74DD958E0C895802D43D931965A95EE
:10017000D1F704C0040404040A111120E4E9F1E0F9
:1001800088E73DD958E0C895802D33D931965A95E6
:10019000D1F704C00E1515040A111120C2D886E843
:1001A00086B980E487B9379AB89AB99ABA9A8A9880
:1001B0008C988B9885B78C7F826085BF7BB7706485
:1001C0007BBF85B7837F886085BF7BB77F777BBF29
:1001D00080E090E0A8E6B0E08D939C93C098C19831
:1001E000C29883E28093C10086E48093C20080E0DD
:1001F00080936A0080E080936B0080E08093BF0072
:1002000080E08093C00080E08093C600929A949A28
:10021000939A839B04C080E08093BE0003C081E07A
:100220008093BE0080E08093C70080E08093C80088
:10023000789402D32AD381E08093C50044D31AD5A1
:100240008FE711E07DD8E8E4F6E165D88FEB11E0A7
:1002500077D8E8E5F6E15FD801D5E3E0F0E072D8C1
:1002600060D88FE711E06CD8EAE6F6E154D884E86C
:10027000C0D8E4E7F6E14FD88FEB11E061D8ECE7A6
:10028000F6E149D8EBD4E3E0F0E05CD8A8E6B0E0D2
:100290000D911C9144E150E0040F151FA3ECB0E058
:1002A0000D931C93A8E6B0E04D915C91A3ECB0E0F7
:1002B0000D911C910417150709F007C0EBD280E0DF
:1002C0008093C500A3ECB0E0C0D70091C50000301A
:1002D00009F01AC00091C700003010F009F001C009
:1002E00013C0DDD281E08093C50080E08093C70019
:1002F000A8E6B0E00D911C9144E150E0040F151FF9
:10030000A3ECB0E00D931C9300916B00003009F05A
:100310001FC007D880916A00D2018C9381E0B6D8C3
:1003200034D2229681E0AED868D4A6E9B0E0EEE8F7
:10033000F6E1BCD8A8E8B0E0E6EBF6E1B7D8B5D274
:1003400081E08093BD006CD4B7D281E080936B00D4
:1003500000916B00013009F00BC00091C700013023
:1003600009F002C0D0D204C0023009F001C001D3AC
:1003700000916B00023009F03FC0E1E0F0E0E2D70D
:1003800073D484EF91E067D86FD484EF91E063D8A1
:100390006BD484EF91E05FD88FE711E0D1D7E4EC24
:1003A000F6E1B9D78FEB11E0CBD7E6EDF6E1B3D7A5
:1003B000E3E0F0E0C7D78FE711E0C2D7E8EEF6E15F
:1003C000AAD78FEB11E0BCD7EAEFF6E1A4D7E3E0C0
:1003D000F0E0B8D780E080936B0080E080936A0003
:1003E000A8E6B0E00D911C9144E150E0040F151F08
:1003F000A3ECB0E00D931C9300916B00033009F067
:10040000A7C0E1E0F0E09ED72FD484EF91E023D89D
:100410002BD484EF91E01FD827D484EF91E01BD830
:100420008FE711E08DD7ECE0F7E175D78FEB11E0A6
:1004300087D7EEE1F7E16FD781E8DBD7E4E2F7E1B8
:100440006AD7E3E0F0E07ED78FE711E079D7E0E309
:10045000F7E161D78FEB11E073D7E2E4F7E15BD707
:10046000E3E0F0E06FD78FE711E06AD7E4E5F7E16A
:1004700052D78FEB11E064D7E6E6F7E14CD781E085
:1004800080936000E3E0F0E05DD780E08093C800F7
:1004900070E87ABF7BB770687BBF8FE711E050D7F9
:1004A000E8E7F7E138D78FEDA4D7ECE7F7E133D7EA
:1004B0008FEB11E045D7EAE8F7E12DD78FED99D71B
:1004C000E0E9F7E128D7E3E0F0E03CD78FE711E07F
:1004D00037D7ECE9F7E11FD78FEB11E031D7EEEA20
:1004E000F7E119D7E3E0F0E02DD70091C700003025
:1004F00081E009F480E08F930091C800013081E031
:1005000009F080E09F91892B882309F409C080E0DD
:100510008093C70080E08093C80080E080936000F3
:1005200000916000003009F0B8CF80E080936A004D
:1005300084E080936B0092D3A8E6B0E00D911C910B
:1005400044E150E0040F151FA3ECB0E00D931C93A1
:1005500000916B00043009F033C08FE711E0F0D652
:10056000E0ECF7E1D8D68FEB11E0EAD6E2EDF7E167
:10057000D2D674D388E29AE06ED78FE711E0E0D646
:10058000E4EEF7E1C8D68FEB11E0DAD6E6EFF7E15B
:10059000C2D681E82ED7EEEFF7E1BDD6E3E0F0E07A
:1005A000D1D680E080936B00A8E6B0E00D911C915D
:1005B00044E150E0040F151FA3ECB0E00D931C9331
:1005C0008B98ACECB0E09C9197FF04C0839B0EC06D
:1005D0009F779C9383990AC089E19F9390E03BD7D2
:1005E0009F91839903C090689C930DD25BCEF89441
:1005F000FFCF0F921F922F923F924F925F927F9266
:10060000AF92BF920F931F932F933F934F935F939C
:100610006F937F938F939F93AF93BF93CF93DF930A
:10062000EF93FF938FB78F938EEE95E89DBD8CBDB2
:1006300088B391E0892788BBA8E6B0E0FFD58F9109
:100640008FBFFF91EF91DF91CF91BF91AF919F91BC
:100650008F917F916F915F914F913F912F911F915A
:100660000F91BF90AF907F905F904F903F902F90F1
:100670001F900F9018950F921F922F923F924F92BA
:100680005F927F92AF92BF920F931F932F933F93EE
:100690004F935F936F937F938F939F93AF93BF938A
:1006A000CF93DF93EF93FF938FB78F930027A0E350
:1006B000B0E08C9182FB00F94427A0E3B0E08C917C
:1006C00084FB40F9041709F004C081E08093C7005F
:1006D00003C082E08093C7008F918FBFFF91EF919D
:1006E000DF91CF91BF91AF919F918F917F916F914A
:1006F0005F914F913F912F911F910F91BF90AF90BC
:100700007F905F904F903F902F901F900F90189583
:100710000F921F922F923F924F925F927F92AF92D1
:10072000BF920F931F932F933F934F935F936F93BA
:100730007F938F939F93AF93BF93CF93DF93EF9369
:10074000FF938FB78F9381E08093C8007BB77F774B
:100750007BBF8F918FBFFF91EF91DF91CF91BF91C1
:10076000AF919F918F917F916F915F914F913F9149
:100770002F911F910F91BF90AF907F905F904F90FE
:100780003F902F901F900F9018958FE711E0D8D5CC
:1007900081E02FD68FEB11E0D3D580E02AD6A88157
:1007A000B9810C91003009F006C08FE712E0C8D57E
:1007B00082E01FD640C0013009F006C08FE712E08A
:1007C000BFD583E016D637C0023009F00BC08FE7E3
:1007D00012E0B6D583E00DD68FEB12E0B1D584E000
:1007E00008D629C0033009F00BC08FE712E0A8D566
:1007F00083E0FFD58FEB12E0A3D585E0FAD51BC0CF
:10080000043009F00BC08FE712E09AD583E0F1D5F0
:100810008FEB12E095D586E0ECD50DC0053009F0E0
:100820000AC08FE712E08CD583E0E3D58FEB12E0AE
:1008300087D587E0DED508950091C1004FE00423FD
:10084000A0E6B0E00C93A0E6B0E08C9180598C93C8
:100850008091C1008093610094E0A1E6B0E034D6BD
:10086000A1E6B0E08C9183708C93A1E6B0E08C910E
:100870008C5A8C9389E2C3D580916000C0D5809159
:100880006100BDD588E2BBD50895A2ECB0E08C91A3
:1008900083BD089580E08093C200F7DF089586E469
:1008A0008093C200F2DFD4D108958FEB14E048D5D5
:1008B000A8E8B0E02AD508958FE714E041D5AAE76B
:1008C000B0E023D5089507B1007F8091C60090E085
:1008D000890F082707B9EFD5A2E6B0E08D939C9366
:1008E000A2E6B0E00D911C910C3B52E0150708F018
:1008F00001C0C19AA2E6B0E08D919C91A6E6B0E05D
:100900008D939C93089580E08093C7008091BD00F3
:1009100081508093BD000091BD00003009F003C0FC
:100920008AE18093BD007CD1C7DFA8E6B0E00D91DD
:100930001C9144E150E0040F151FA3ECB0E00D93AF
:100940001C930091BE00013009F012C0AFEBB0E083
:100950008C918F5F8C930091BF00053010F009F0EF
:1009600001C006C080E08093BF0080E08093BE009D
:10097000089580E08093C700ADEBB0E08C918F5F6D
:100980008C930091BD000B3109F003C081E080938E
:10099000BD0046D191DFA8E6B0E00D911C9144E185
:1009A00050E0040F151FA3ECB0E00D931C930091D1
:1009B000BE00013081E009F080E08F930091BF001C
:1009C000053081E009F080E09F918923882309F4B4
:1009D00013C0A0ECB0E08C918F5F8C930091C000AD
:1009E000053010F009F001C006C080E08093C0001F
:1009F00080E08093BE0006C080E08093C00080E06D
:100A00008093BE0008950091C500003009F005C034
:100A100046DF81E08093C500EFC00091BE00013049
:100A200009F038C00091BF00053081E009F080E096
:100A30008F930091C000053081E009F080E09F9124
:100A40008923882309F41CC083E080936B00AAECFF
:100A5000B0E0F4D3E1E0F0E0AAECB0E07BE7C8D589
:100A600060D48FE711E06CD4E8E0F8E154D48FEB68
:100A700011E066D4A0E5B3E0EAECF0E048D543D459
:100A800080E08093BE0080E08093BF0080E0809390
:100A9000C000A6C0009180000A3209F4A1C080E025
:100AA0008093610081E080936000009160000D30D0
:100AB00010F009F023C040918000A0E6B0E0AD90B6
:100AC000BB24ABE6B0E0AA0DBB1D0C91041709F0E6
:100AD0000EC081E08093610080918000A0E6B0E0CC
:100AE000AD90BB24A7E8B0E0AA0DBB1D8C93A0E697
:100AF000B0E08C918F5F8C9308F4D7CF00916100A8
:100B0000013009F007C0D1DEA3D084E690E0A3D481
:100B10009FD01EC0AAE6B0E08C918F5F8C9380912D
:100B20006A00D2018C9381E0B1D42FDE229681E05D
:100B3000A9D400916A00053009F009C082E08093D1
:100B40006B00ECE6F0E0A8E8B0E036D5AEDE8CD085
:100B50000091800040E2040FA1E6B0E00C9381E038
:100B60008093600000916000063210F009F01FC011
:100B700040916100A0E6B0E0AD90BB24A5E9B0E0F3
:100B8000AA0DBB1D0C91041709F00AC080E2A0E673
:100B9000B0E0AD90BB24A5E9B0E0AA0DBB1D8C93DD
:100BA000A0E6B0E08C918F5F8C9308F4DBCF38D057
:100BB00083DEECE6F0E0A8E8B0E035D581E009F0AE
:100BC00080E08F9300916A00053081E008F080E0BA
:100BD0009F918923882309F403C083E080936B00ED
:100BE000A8E6B0E00D911C9144E150E0040F151F00
:100BF000A3ECB0E00D931C93089584E690E08A93F3
:100C00009A9331D3A0E6B0E00C93E4ECFCE0A0E6CC
:100C1000B0E08C91992764D4ACE6B0E047D4089555
:100C20008091BD00E6E9F0E00DE00A93AAE7B0E0AC
:100C3000C8D400918000003209F406C0A0E8B0E0FA
:100C40008C9180528C9303C08AE280938000089537
:100C5000C29A84E690E0FFD3C2980895C29A80E9D0
:100C600091E0F9D3C2980895C29AE1E0F0E06AD326
:100C7000C2980895E0E0F0E0A9ECB0E0C8D400919B
:100C8000C900013009F416C081E08093C90080E0FA
:100C900090E0AAECB0E08D939C93E1E0F0E0AAEC48
:100CA000B0E07BE7A5D4E0E0F0E0A9ECB0E07BE7C2
:100CB0009DD405C0E1E0F0E0AAECB0E0AAD408952C
:100CC000F894FFCF57454C545241554D4641485238
:100CD00054004142454E54455545524C4943480005
:100CE0004142454E54455545524C55535400414E92
:100CF0004C4147454F424A454B544500415354529D
:100D00004F47454F4C4F47494500415354524F427E
:100D1000494F4C4F47494500424552474B52495372
:100D200054414C4C45004245524753544154494F5D
:100D30004E454E004245524753544549474552455A
:100D400049004245524757414E444552554E47008F
:100D50004D59535445525943414348455300484126
:100D6000555341504F5448454B454E00484155530B
:100D700056455257414C54455200484155534841FD
:100D80004C545357415245004645535453504945DE
:100D90004C484155530046414C53434841555353E9
:100DA00041474500574F4348454E454E44484155FD
:100DB00053004841555342455345545A554E4700F8
:100DC0005741434B454C4B4F4E54414B54005741B8
:100DD000434854454C5343484C41470046414852D0
:100DE00052414446414852454E00445552434847BB
:100DF000454C415546454E0041535048414C5443A3
:100E00004F57424F5900415242454954535A494D58
:100E10004D45520046455545525745485241555457
:100E20004F004142534348494544534B55535300A7
:100E300042554E4445534B414E5A4C4552005A5729
:100E4000494542454C534348414C450042414E4B75
:100E500047454845494D4E495300414E5349434843
:100E600054534B4152544500415354524F504859EA
:100E700053494B4552004645554552574548524DFA
:100E8000414E4E004B414C454E4445524D4F4E4114
:100E90005400484146454E4152424549544552004E
:100EA000434F4D50555445524649524D41004B4ECB
:100EB0004F424C415543485A454845004C455543DF
:100EC000485452454B4C414D45004D494E555445B3
:100ED0004E5A454947455200564552535445434B97
:100EE000535049454C00414D454953454E484155A5
:100EF00046454E004B41504954414C414E4C4147B0
:100F0000450047414E47534348414C54554E4700D6
:100F10004D55545445525350524143484500424563
:100F20005255465342455241544552004E45424562
:100F30004C534348574144454E004F424552494E59
:100F40005350454B544F520057415343484D415322
:100F50004348494E4500424C554D454E5343484D3C
:100F600055434B004F5249454E5454455050494308
:100F7000480044414D50464D41534348494E450079
:100F8000504552534F4E454E574147454E00504FE6
:100F90004C495A454953434855545A0046414D49D6
:100FA0004C49454E4E414D454E00524153494552E4
:100FB000415050415241540053415454454C5441C6
:100FC000534348454E005A415050454C5048494CB7
:100FD000495050005441534348454E4D45535345A5
:100FE0005200494445454E524549434854554D00E9
:100FF000544F4445534B414E4449444154004B41A6
:101000004E4F4E454E465554544552004745495360
:101010005445525354554E444500554D5354414E3A
:1010200044534B4C45494400494E4E454E4D494E64
:101030004953544552005241554D464F525343482F
:10104000554E4700554E5445524F4646495A49451C
:101050005200434F4D5055544552535049454C0052
:1010600056414E494C4C455343484F544500504F10
:101070004C544552474549535445520056455253E6
:1010800055434853524549484500454C454B5452F9
:101090004F4D41474E45540057414C4E5553534BCD
:1010A000554348454E00534348415454454E424FE2
:1010B00058454E004841555054534348414C5445BF
:1010C00052005A494D4D4552414E54454E4E4500F1
:1010D0005741535345524C454954554E470045528C
:1010E00044554D4C4155464241484E005A5547568D
:1010F000455242494E44554E470045494E54524987
:1011000054545347454C4400574152544553434867
:101110004C414E4745005A55434B45524D454C4F67
:101120004E454E00454E45524749455155454C4C5C
:1011300045005741535345525350494547454C008C
:101140005645524B454852534348414F5300454E34
:101150004552474945424544415246005343484D54
:1011600045525A4D495454454C00564552424F54ED
:1011700053534348494C44004E494544524947570C
:101180004153534552004641485252414452454909
:1011900046454E0054524F4D4D454C4252454D53DD
:1011A000450053434841554B454C535455484C001A
:1011B000494E465241535452554B54555200524594
:1011C0004348454E4155464741424500504F4C49E2
:1011D0005A454957414348454E005A41484C454EAF
:1011E0005343484C4F5353004D4F4445494E44558B
:1011F0005354524945004C49434854534348414C89
:10120000544552004252494546554D5343484C417E
:1012100047004B4C415353454E5A494D4D455200A2
:10122000484155544155535343484C414700494E5A
:1012300053454B54454E504C41474500ED91FC9170
:10124000EF5FFF4FFC93EE930895ED91FC91E15019
:10125000F040FC93EE93089515E000E000936600E3
:1012600010936700089540916600509167000DEF5C
:1012700013E412D10D5311460093660010936700DA
:101280005991499126D0089508D006D100FC10D07C
:10129000089503D01ED001F8F9CF0024E89457FF39
:1012A00002C009D0689400F80BD010F8012408950A
:1012B00002D009D00895509540954F5F5F4F089533
:1012C000E89417FF0895009510950F5F1F4F6894DD
:1012D0000895352F242FE894452B11F46894089530
:1012E000512F402F0027112780E1440F551F001F69
:1012F000111F021B130B416018F4020F131F4E7FC6
:101300008A9599F70895A0E5B3E08D91882311F0AF
:1013100070D0FBCF0895E0D0802D11F06AD0FBCFC4
:10132000089581E06CD014D080E869C08FE7213047
:1013300039F08FEB223021F08FE8233009F08FEC69
:10134000810F5DC088EE93E086D03197D9F708957C
:1013500083E0992780C08AEF90E07DD0A59AA49A77
:10136000A39AA29A8E9A8F9A979885E090E073D06C
:101370009698AD98AC98AB9AAA9A969AEF93FF93E9
:10138000E4ECF0E05CD0FF91EF91969861D0969AF2
:10139000EF93FF93E4ECF0E052D0FF91EF91969839
:1013A00057D0969AEF93FF93E4ECF0E048D0FF918A
:1013B000EF9196984DD0AA98969AEF93FF93E4EC0C
:1013C000F0E03DD0FF91EF91969842D089E217D09E
:1013D0008CE115D082E513D089E611D084E70FD0D7
:1013E00088E20DD088E20BD08EE009D086E007D0ED
:1013F0000895979A829505D004D02AD00895979899
:10140000F9CF859510F4AA9A01C0AA98859510F491
:10141000AB9A01C0AB98859510F4AC9A01C0AC981A
:10142000859510F4AD9A01C0AD98969AEF93FF930D
:10143000E4ECF0E004D0FF91EF9196980895319795
:10144000F1F70895689462F80895E89462F80895B1
:1014500081E090E000C0EF93FF93EE27E82BE92BAB
:1014600031F0E0EDF7E03197F1F70197D1F7FF9117
:10147000EF91089501911191219130810895481AB9
:10148000590A0895481A8827580A089599275A92A0
:101490004A92480E591E08950F92B801469F800146
:1014A000479F100D569F100D0F90089515D00D9267
:1014B0000020E1F70895369A3699FECF369A36998C
:1014C000FECF84B195B10895903029F08C91869526
:1014D0009A95E9F78C930895C89531960020089560
:1014E000882311F4992321F0F7DFF1F70197E1F751
:1014F0000895000F111F221F331F089500951095A6
:10150000209530950F5F1F4F2F4F3F4F089501914A
:1015100010810BC0AFDF0BC00191108117FF05C018
:101520003FEF2FEF04C0008111272227332737FF19
:1015300003C0E4DF8DE28D93CF92DF92EF92AA2475
:10154000BB24CC24DD24EE2440E2EAE0FF2755E072
:1015500093E38081890F87FD9F7083FD907F891BB6
:1015600081935A95A9F7C5DFAA1CBB1CCC1CDD1CB6
:10157000EE1C4A9551F7E894EFE0FF2782910CD0DA
:10158000EB30E0F71EF068948A2D0AD088278D93FF
:10159000EF90DF90CF900895982F829501D0892FFA
:1015A0008F70805D26F0803309F4089568948D93E0
:1015B000089588278D93089581918D938823E1F76D
:1015C000089509919191992351F08A95D9F731970E
:1015D00081918D930A9519F08823D1F70895E9CF69
:1015E000E199FECFEEBBFFBB3196089591E001C0BB
:1015F00092E07B3751F47FB7F894F2DF8D918DBB89
:10160000E29AE19A9A95C9F77FBF7727089591E00A
:1016100001C092E0E5DFE09A8DB38D939A95D1F702
:101620000895689401C0E894AF93BF938D9116F02C
:10163000919102C051DF902D891718F011F4882381
:10164000A9F7BF91AF9108952057696C6C6B6F6DCE
:101650006D656E207A756D0047656F6361636869BB
:101660006E6720537069656C00002047616C676588
:101670006E6D00006E6E6368656E00002020202095
:10168000204743353835424D202020200000757614
:101690007778797A6162636465666768696A6B6C9A
:1016A0006D6E6F707172737475767778797A616226
:1016B0006364656600005F5F5F5F5F5F5F5F5F5FE2
:1016C0005F5F5F00212121202053636861646520F2
:1016D0002021212100004C65696465722020766517
:1016E000726C6F72656E000050726F626965726530
:1016F00020657320646F6368000065696E666163CE
:1017000068206E6F63686D616C7300002121204852
:1017100065727A6C696368656E2021210000212062
:1017200020476C00636B77756E736368202100003F
:1017300044752068617374206765776F6E6E656E9F
:101740000000756E642066696E646573742064655C
:101750006E20000043616368652062656920666FE2
:101760006C2D2020000067656E64656E204B6F6FE6
:101770007264732E2E2000004E3438002033312E38
:101780003233352020202020000045303039000041
:101790002035342E3839392020202000526F6872CD
:1017A00020756E74657220537465696E0000756EE5
:1017B000642057656720766F6E206F62656E00004B
:1017C0004F6B204475206D6167737420616C736F7B
:1017D00000006E6F63686D616C20737069656C6585
:1017E0006E2100004E612064616E6E206C6F73206C
:1017F000756E642000007669656C20476C00636B31
:101800002121212121210000427970617373636FCE
:08181000756E7465723A000068
:00000001FF
